:100000000C94EC010C9409020C9409020C94090262
:100010000C9409020C9409020C9409020C94090234
:100020000C9409020C941D0B0C9409020C94090207
:100030000C94D6140C9409020C9409020C94090235
:100040000C9409020C9409020C94590A0C940902AC
:100050000C9451040C9409020C941B040C94090296
:100060000C94030C0C9409020C940B140C940902CC
:100070000A0A0D004E65757472616C004865616412
:10008000696E67486F6C64000A0D5374657565721C
:10009000756E673A20004F4B0A0D000A0D416267EA
:1000A0006C65696368204C756674647275636B7304
:1000B000656E736F722E2E000A0D42656E75747A2E
:1000C0006520506172616D657465727361747A2028
:1000D0002564000A0D496E69742E20454550524F23
:1000E0004D3A2047656E65726965726520446566A4
:1000F00061756C742D506172616D657465722E2E20
:100100002E000A0D3D3D3D3D3D3D3D3D3D3D3D3DCE
:100110003D3D3D3D3D3D3D3D3D3D3D3D3D3D3D3D0F
:100120003D3D000A0D466C69676874436F6E7472DA
:100130006F6C0A0D48617264776172653A25642EAE
:1001400025640A0D536F6674776172653A562564AB
:100150002E256420002E0052616E67653A253369B2
:100160002D253369005374656C6C756E673A2025D4
:10017000336900536574706F696E7420202533698C
:1001800000536572766F202000506F7469343A20F6
:100190002025336900506F7469333A202025336974
:1001A00000506F7469323A202025336900506F7413
:1001B00069313A20202533690053746172743A2002
:1001C00020202020253569004D6573737765727492
:1001D0003A2020253569005269636874756E673A64
:1001E0002020253569004B6F6D70617373202020CE
:1001F0002020202000456D70662E506567656C3AA2
:10020000253569005370616E6E756E673A20202542
:10021000356900486F6368202534692028253369D3
:100220002900526F6C6C20253469202825336929F8
:10023000004E69636B202534692028253369290025
:10024000414343202D2053656E736F7200476965EB
:10025000722025346920282533692900526F6C6C7F
:1002600020253469202825336929004E69636B20D5
:10027000253469202825336929004779726F202D9C
:100280002053656E736F720050333A253469202015
:1002900050343A253469200050313A253469202001
:1002A00050323A253469200047733A2534692020BA
:1002B00047693A25346920004E693A25346920207F
:1002C000526F3A25346920004B373A253469202093
:1002D0004B383A25346920004B353A2534692020C3
:1002E0004B363A25346920004B333A2534692020B7
:1002F0004B343A25346920004B313A2534692020AB
:100300004B323A25346920004B6F6D706173733A3C
:1003100020202025356900526F6C6C3A2020202067
:100320002020253569004E69636B3A20202020206B
:100330002025356900616B742E204C61676500488B
:10034000F668656E726567656C756E67004B65690A
:100350006E6520004F66662020202020203A202550
:100360003569004C756674647275636B3A20253587
:100370006900536F6C6C486F6568653A2025356974
:1003800000486F6568653A202020202025356900E7
:1003900028632920486F6C6765722042757373006B
:1003A00053657474696E673A202564200048573A93
:1003B0005625642E25642053573A25642E25640063
:1003C0002B2B204D696B726F4B6F70746572202BF5
:1003D0002B005B25695D000011241FBECFEFD0E12B
:1003E000DEBFCDBF11E0A0E0B1E0E8E3FAE502C076
:1003F00005900D92A039B107D9F715E0A0E9B1E059
:1004000001C01D92A333B107E1F70E9448020C948A
:100410001B2D0C94000022E030E0D9010E94072D32
:10042000802D863028F082E0D901082E0E940F2D01
:1004300099270895FB01282F863008F025E0842FA6
:100440009927429FD0011124AC59BF4F019724F046
:1004500001900E940F2DFACFA2E0B0E0022E0E9480
:100460000F2D0895CF93DF93FB01C42FDD27863036
:1004700008F085E0489FD0011124AC59BF4F219767
:1004800024F00E94072D0192FACFDF91CF910895B9
:100490001F93CF93DF93189B02C08BE001C08AE0CB
:1004A0008093000181E887B98FEF88B98BE184B927
:1004B00081E085B98EE38AB9579A87EF8BB984B703
:1004C000877F84BF80916000886180936000109274
:1004D000600080ED97E09093AD018093AC011092A5
:1004E0002D0210922C021092BC041092BB041092A8
:1004F0002B0210922A021092290210922802809157
:1005000000018A3011F4289801C0289A0E94C40B77
:100510000E9423060E94C1140E94FD0B0E94F11349
:1005200078941092BA038FE38093BB0385E08093A5
:10053000BC03209100018FE390E09F938F931F9263
:100540001F92822F6AE00E94972C892F99279F93F0
:100550008F93822F0E94972C99279F938F9383E2EA
:1005600091E09F938F931F920E94B70782E091E0E2
:100570009F938F931F920E94B707299AA1E0B0E042
:100580000E94072D802D2DB73EB7225F3F4F0FB63B
:10059000F8943EBF0FBE2DBF8E33A9F183ED90E0DE
:1005A0009F938F931F920E94B7070E947C1C4AE37F
:1005B00063EE74E080E00E941A0211E00F900F9049
:1005C0000F90123049F40E94051C4AE363EE74E078
:1005D00082E00E941A0213E04AE363EE74E0812F86
:1005E0000E941A021F5F163060F382E022E030E0C2
:1005F000D901082E0E940F2D8EE321503040D901E1
:10060000082E0E940F2DC2E0D0E0DE010E94072DCF
:10061000802D863028F082E0DE01082E0E940F2D0A
:100620004AE363EE74E00E943202DE010E94072D6D
:10063000802D863028F082E0DE01082E0E940F2DEA
:1006400099279F938F9388EB90E09F938F931F92AE
:100650000E94B7078091EB040F900F900F900F90BE
:100660000F9080FF20C08BE990E09F938F931F92A3
:100670000E94B70788EE93E00E94080BEC010E94ED
:10068000BF0F0F900F900F90CE010E94110B882387
:10069000D9F386E990E09F938F931F920E94B7074A
:1006A0000F900F900F900E943A1D809100018A30A8
:1006B00011F4289801C0289A80ED97E09093AD013D
:1006C0008093AC0188EE93E09093B5038093B403DC
:1006D00085E58093AF0388E890E09F938F931F9206
:1006E0000E94B7078091EB040F900F900F9082FF4C
:1006F00003C08CE790E002C084E790E09F938F9363
:100700001F920E94B7070F900F900F9080E790E024
:100710009F938F931F920E94B7070E94031088E84F
:1007200093E190937B0180937A010F900F900F904B
:100730008091A901882309F451C01092A9010E9457
:10074000851E0E94F31C209100012A3011F4289884
:1007500001C0289A80910201882319F0815080936A
:10076000020180912702882329F08091270281507D
:100770008093270280917A0190917B01892B01F56A
:1007800085E090E090937B0180937A010E949B1416
:1007900080910301909104018F5F9F4FF9F4809144
:1007A0002E028823D9F080E197E29093AD018093E7
:1007B000AC0180E890E090930401809303010EC0A7
:1007C00080917A0190917B01019790937B018093B6
:1007D0007A012A3011F4289801C0289A0E943E0616
:1007E0000E94B406CE010E94110B882309F4A0CF09
:1007F00020910701309108018091FB049927281767
:1008000039079CF480910301909104018F5F9F4F01
:1008100061F480E797E19093AD018093AC0180E0B3
:1008200093E0909304018093030184E690E00E949A
:10083000080BEC017DCF1F920F920FB60F9211247F
:100840008F939F93EF93FF93809101018823E1F4AD
:100850008091A5019091A60101969093A6018093A5
:10086000A501FC01EF57FD4FE081ED3019F086390D
:10087000910539F41092A6011092A50181E08093B0
:100880000101E093C60004C01092A6011092A501D8
:10089000FF91EF919F918F910F900FBE0F901F903E
:1008A00018951F920F920FB60F9211242F933F931A
:1008B0004F938F939F93AF93BF93CF93DF93EF9318
:1008C000FF938091C600809394014091A001463926
:1008D00010F010929F01809194018D3009F05CC05E
:1008E00080919F01823009F057C010929F01A42F80
:1008F000BB27FD01EE53FC4F3081ED01CD53DC4FA2
:1009000028818091A3019091A401831B9109821BEE
:1009100091099F709093A4018093A3019C0196E09C
:10092000369527959A95E1F7235C2093A201982F9D
:100930009F73935C9093A1018081281729F488818B
:10094000981711F491E006C0809197018F5F809312
:10095000970190E080919501882309F064C0992364
:1009600009F461C081E08093950140939801AC53F4
:10097000BC4F8DE08C938091C603823509F053C043
:1009800088E190E02CE00FB6F894A8958093600081
:100990000FBE2093600047C080919F018130D9F045
:1009A000813018F08230E9F530C0809194018332B3
:1009B00039F480919501882319F481E080939F0197
:1009C000809194018093C40381E08093A001809181
:1009D0009401992715C082E080939F01E42FFF279F
:1009E00080919401EC53FC4F80834F5F4093A001B2
:1009F000209194018091A3019091A401820F911DF7
:100A00009093A4018093A3010EC0E42FFF2780914F
:100A10009401EC53FC4F8083463938F310929F01C8
:100A2000E7CF10929F01FF91EF91DF91CF91BF919E
:100A3000AF919F918F914F913F912F910F900FBE4A
:100A40000F901F901895DC0120E030E040E050E06E
:100A5000E1E8F2E005C08191280F311D4F5F5F4F43
:100A60004A175B07C1F73F70C90136E09695879535
:100A70003A95E1F7835CFD01EF57FD4F80831196B6
:100A80002F73235CFD01EF57FD4F2083AE57BD4F01
:100A90008DE08C9310920101809181028093C600B9
:100AA0000895EF92FF920F931F93CF93DF937A01F4
:100AB000722F93E29093810260938202809383026B
:100AC00003E010E060E0A4E8B2E046C0F701E60F02
:100AD000F11D90816F5F715019F4E0E040E00FC0AC
:100AE000F701E60FF11D40816F5F715011F4E0E0F6
:100AF00006C0F701E60FF11DE0816F5F7150892F8D
:100B000086958695835C8C935527892F99278370CA
:100B1000907024E0880F991F2A95E1F79A0194E0DC
:100B2000369527959A95E1F7822B835CED018983B1
:100B30004F705070440F551F440F551F8E2F8295D4
:100B4000869586958370842B835C8A83EF73E35C40
:100B5000EB830C5F1F4F1496772309F0B7CFC801C2
:100B60000E942305DF91CF911F910F91FF90EF908D
:100B700008951F93CF93DF93EC0170E0A22FBB2762
:100B8000129748C0E42FFF27EC53FC4F30814F5F92
:100B9000E42FFF27EC53FC4F50814F5FE42FFF27DA
:100BA000EC53FC4F10814F5FE42FFF27EC53FC4FB9
:100BB00020814F5F842F9927A817B90774F15D53DF
:100BC000FE01E70FF11D3D53330F330F852F829543
:100BD0008F70382B3083613001F1912F9D537F5FEF
:100BE000FE01E70FF11D71505295507F892F8695B8
:100BF0008695582B508363506F3F79F07E5FFE01DE
:100C0000E70FF11D9295990F990F907C2D53922B20
:100C100090837F5F662309F0B5CFDF91CF911F915D
:100C200008951F93182F8A3019F48DE00E94110641
:100C30008091C00085FFFCCF1093C60080E090E05B
:100C40001F9108950895E1ECF0E088E18083A0EC25
:100C5000B0E08C9182608C938081806880838081F9
:100C6000806480838AE28093C40088EC90E00E94D4
:100C7000080B9093AE038093AD030895809101011A
:100C8000882309F470C080919001882371F08091CD
:100C90000101882351F02BE04FEA53E0609180027C
:100CA00087E40E945105109290018091AD039091CC
:100CB000AE030E94110B882321F4809192018823B6
:100CC000B1F080910101882391F022E44AE554E0DB
:100CD0006091800284E40E9451051092920184EF99
:100CE00091E00E94080B9093AE038093AD03809136
:100CF0009101882331F180910101882311F10E9433
:100D00000C101092910180919E01982F9F5F9093FB
:100D10009E01943059F426E147EB54E060E084E30F
:100D20000E9451058FEF80939E010BC044E1949F78
:100D3000A0011124475E5E4F24E160E08F5C0E94B9
:100D4000510580919301882371F0809101018823DE
:100D500051F02AE04AEB53E06091800286E50E9460
:100D600051051092930108951F93CF93DF93CDB750
:100D7000DEB722970FB6F894DEBF0FBECDBF8091CD
:100D80009501882309F490C08FEF80930201809130
:100D9000C603813758F48C3608F067C08736C9F12E
:100DA0008836C1F0833609F07DC008C0843721F150
:100DB000863759F1813709F075C02FC0209198010D
:100DC00043E06BE08FEA93E00E94B90581E08093F5
:100DD000920168C02091980143E062E0CE01019643
:100DE0000E94B9058091CE019981892B8093CE0113
:100DF00081E08093910156C02091980143E064E026
:100E00008AE991E00E94B9054DC081E08093930189
:100E100049C081E08093900145C02091980143E052
:100E200062E0CE0101960E94B90589818F3F89F069
:100E3000863010F085E089834AE363EE74E08981AF
:100E40000E94320289812AE343EE54E060918002DD
:100E500008C0109180020E940B022AE343EE54E086
:100E6000612F855B0E9451051DC02091980143E0D0
:100E70006AE383EE94E00E94B9058091C6034AE3D9
:100E800063EE74E08B560E941A028091C6038B5663
:100E9000A2E0B0E0082E0E940F2D0E940B029927BD
:100EA0000E94701E1092950122960FB6F894DEBF34
:100EB0000FBECDBFDF91CF911F910895982F8091E4
:100EC0009C04813069F48091CD01E82FFF27E75E13
:100ED000FE4F90838F5F8093CD0121E030E005C00D
:100EE000892F0E941106282F3327C90108951F93C7
:100EF000182F04C080E30E945E0711501116D4F32E
:100F00001F9108951F93182F04C080E20E945E076E
:100F100011501116D4F31F9108950F931F93CF937F
:100F2000DF938C01EB0108C0F8010F5F1F4FE491C4
:100F30008E2F0E945E0721972097B1F7DF91CF9106
:100F40001F910F9108950F931F93CF93DF938C01FF
:100F5000EB0106C0F80181918F010E945E07219785
:100F60002097C1F7DF91CF911F910F9108952F9294
:100F70003F924F925F926F927F928F929F92AF9229
:100F8000BF92CF92DF92EF92FF920F931F93CF9376
:100F9000DF93CDB7DEB7E3970FB6F894DEBF0FBE91
:100FA000CDBF29968FAD299780939C04CE01855B98
:100FB0009F4F9D838C832B968EAD9FAD2B979FA7C4
:100FC0008EA722243324210102C0130124010EA57F
:100FD0001FA502C00F5F1F4FF801F490FF2019F00A
:100FE000F5E2FF16B9F7B8018EA59FA5681B790B2E
:100FF00011F00E948D07FF2009F442C20F5F1F4FBE
:101000001FA70EA71982AC81BD811BAA1AAA9FEF48
:1010100099ABEEA5FFA5CF0101969FA78EA7B4902F
:1010200095E7B91621F08B2D8062883789F4EBA9FA
:10103000E0FF07C02D903D904D905C901397149663
:1010400007C08D919C9111971C0144245524129640
:10105000F0E2BF1621F489818823D9F685C083E2A6
:10106000B81609F483C09AE2B91621F0EDE2BE1673
:1010700069F408C0FD011296E081EAABE7FFC9CF31
:10108000E195EAABFBA9F061FF7D72C08BE2B81677
:1010900009F46AC09EE2B916B1F52EA53FA52F5FEF
:1010A0003F4FEEA5FFA584918A3221F0B82E20E0B3
:1010B00030E01BC0FD0112964081518157FF02C0F4
:1010C0004FEF5FEF49AB3FA72EA7A3CFC90103E0C6
:1010D000880F991F0A95E1F7220F331F280F391F38
:1010E0002B0D311D20533040B49031968B2D805301
:1010F0008A3060F3FFA7EEA7A90137FF02C04FEFC8
:101100005FEF49AB8DCFF0E3BF1631F48BA984FDBF
:1011100080CF80628BAB7DCF8B2D81538930E8F4FB
:1011200020E030E0C901F3E0880F991FFA95E1F75C
:10113000220F331F280F391F2B0D311D2053304034
:10114000EEA5FFA5CF0101969FA78EA7B4908B2D8A
:1011500080538A3038F32AAB63CF98E6B91651F43E
:10116000EBA9E460EBAB55CFB98253CFFBA9F86094
:10117000FBAB4FCF8CE6B81621F49BA991609BABDB
:1011800048CFBD83AC83E3E6BE1639F41296BD8327
:10119000AC8312978C918E8318C1F4E4BF1639F09A
:1011A00084E6B81639F099E6B91659F503C0EBA9EB
:1011B000E160EBABFBA9F0FF08C01496BD83AC83E4
:1011C0005E904E903E902E900AC01296BD83AC83E6
:1011D0009E918E911C01442437FC4094542C57FC62
:1011E00003C08AE088AB92C050944094309420941D
:1011F000211C311C411C511C8DE289839AE098AB63
:1012000085C0EFE4BE1629F0FFE6BF1639F488E08A
:1012100061C09BA991609BABE8E056C0F0E7BF16A8
:1012200071F41296BD83AC839E918E911C0144246F
:1012300055248BA980648BAB78E7B72E5EC0E3E7BB
:10124000BE16D9F51296BD83AC83DE90CE90C11444
:10125000D10489F488E28E838EE68F8385E78887C0
:101260008CE689878A8789E28B871C8666E0C62E92
:10127000D12CCC0EDD1EF9A9F7FD13C04F2F552739
:1012800047FD509560E070E0C6010E94032B009777
:1012900011F419A90DC08C1919A981174CF4182F34
:1012A00007C0F60101900020E9F731971E2F1C19A5
:1012B00019824201310140E094C085E5B81631F051
:1012C00095E7B91649F4EAE0E8AB1FC0FBA9F16065
:1012D000FBAB8AE088AB19C098E5B91621F0E8E7C6
:1012E000BE1609F06EC0FBA9F3FD02C080E1F2CF8B
:1012F000211431044104510419F490E198AB05C064
:10130000EBA9E064EBABF0E1F8AB198289A987FDAA
:1013100003C09BA99F7D9BAB211431044104510460
:1013200061F4E9A9EE2349F46624772443015EE2DF
:10133000C52ED12CCC0EDD1E3EC04EE2C42ED12CCB
:10134000CC0EDD1EF8A9EF2EFF2400271127C201C5
:10135000B101A80197010E94CA2C6A3020F430E341
:10136000A32EA60E08C027E5A22EA60E88E5B81665
:1013700011F49FEDA922F601A2926F01C201B10101
:10138000A80197010E94CA2C39014A012E143F047A
:101390004006510618F019012A01D9CFF8A9F830F2
:1013A00051F48BA983FF07C090E3A91621F080E3D5
:1013B000F60182936F01CE018C19182F125D49A995
:1013C00010C0BB2009F45CC0BE8219824201310109
:1013D00000E096E0C92ED12CCC0EDD1E11E021E0FC
:1013E00005C0212F042F011B07FD00E08981882300
:1013F00019F0812F8F5F07C09BA996FD02C0812F36
:1014000002C0822F8E5FA82EA00EEBA9EE2EFF2425
:1014100080E3482E512C4E205F204114510421F4CA
:101420008AA98A190E9482078981882329F061E0AC
:1014300070E0CE01019609C0E6FE09C080E38A8310
:10144000BB8262E070E0CE0102960E94A307F0E248
:101450004F16510421F48AA98A190E947707802F18
:101460000E947707612F772767FD7095C6010E945C
:10147000A307E4FEAACD8AA98A190E948207A5CDF6
:10148000E3960FB6F894DEBF0FBECDBFDF91CF91CC
:101490001F910F91FF90EF90DF90CF90BF90AF9092
:1014A0009F908F907F906F905F904F903F902F9084
:1014B00008951F920F920FB60F9211242F933F930E
:1014C0005F936F937F938F939F93AF93BF9380911D
:1014D000B00181508093B0018F3FB9F489E08093CF
:1014E000B001809106018F5F81708093060188238F
:1014F00019F481E08093A9018091A7019091A8013E
:1015000001969093A8018093A7018091AC019091DE
:10151000AD010297B8F08091AC019091AD010197B7
:101520009093AD018093AC018091AC019091AD019D
:10153000209103013091040182239323892B09F028
:1015400053C006C08FEF9FEF909304018093030177
:10155000809100018A3039F404C05A9A05C0479A34
:1015600003C05A9801C047988091EB0483FF42C0A2
:10157000349B0AC08091AA019091AB01019690938F
:10158000AB018093AA0136C08091AA019091AB0172
:10159000892B79F08091AA019091AB01805A9F40EC
:1015A00040F48091AA019091AB019093180280932E
:1015B0001702809117029091180220911902309120
:1015C0001A02821B930B845E9D4F68E671E00E94B5
:1015D000B72C845B904090931C0280931B02109266
:1015E000AB011092AA0106C0809100018A3009F077
:1015F000B6CFB3CFBF91AF919F918F917F916F91F4
:101600005F913F912F910F900FBE0F901F901895F3
:101610002091A7013091A8012F5F3F4F820F931FA8
:1016200008952091A7013091A801821B930B892F67
:10163000992786958074992708951F920F920FB667
:101640000F921124EF92FF920F931F932F933F93CA
:101650004F935F936F937F938F939F93AF93BF93BA
:10166000CF93DF93EF93FF93809105018150809397
:1016700005018F3F09F06DC083E88093B000809131
:101680008D01C82FDD27D093AF01C093AE018091AB
:101690000C05E090050580FF1EC06091E701709188
:1016A000E8018091E9019091EA01FF2400271127C8
:1016B00020E830E040E050E00E94EC2CC801B70187
:1016C0000E94782C20E032E040E050E00E94EC2CB8
:1016D000C20FD31F1DC06091E7017091E801809196
:1016E000E9019091EA01FF240027112720E830E06A
:1016F00040E050E00E94EC2CC801B7010E94782C19
:1017000020E032E040E050E00E94EC2CC21BD30B02
:10171000D093AF01C093AE012091AE013091AF01E3
:101720008091060599272817390734F0809107051D
:1017300099278217930724F49093AF018093AE0109
:101740008091AE018093B3008091080580930501DC
:1017500004C083E08093B0005F98FF91EF91DF9128
:10176000CF91BF91AF919F918F917F916F915F9139
:101770004F913F912F911F910F91FF90EF900F90FC
:101780000FBE0F901F9018958091A7019091A8010E
:101790000B969093B2018093B10182E085BD83EAFC
:1017A00084BD17BC88E788BD96E096BD83EC809326
:1017B000B0009093B100E0E7F0E080818260808328
:1017C000EEE6F0E08081816080838AE08093B30060
:1017D0001092B20008952091A7013091A8012F5FC7
:1017E0003F4F280F391F8091A7019091A801A901AF
:1017F000481B590B57FFF7CF089510927C008FEECE
:1018000080937A0008951F920F920FB60F921124C1
:10181000EF92FF920F931F932F933F934F935F93FA
:101820006F937F938F939F93AF93BF93CF93DF93E8
:10183000EF93FF9310927A004091C9014F5F40935C
:10184000C9014150433009F4B4C1443038F4413047
:1018500009F469C0423008F008C10DC0453009F4F0
:10186000E8C1453008F4C2C1463009F407C2473028
:1018700009F063C3EAC22091DB013091DC01809161
:10188000780090917900281B390B809100018A30F3
:1018900011F0220F331F8091B7019091B801820F90
:1018A000931F9093B8018093B7018091C1018F5F1E
:1018B0008093C10180910B0290910C02A0910D02C6
:1018C000B0910E02442737FD4095542F820F931F8D
:1018D000A41FB51F80930B0290930C02A0930D02DE
:1018E000B0930E0280910F0290911002A09111020C
:1018F000B0911202820F931FA41FB51F80930F0295
:1019000090931002A0931102B093120281E0809391
:10191000CA018091C7019091C80101969093C801B6
:101920008093C7010EC36091780070917900809117
:10193000D9019091DA01681B790B809100018A30FE
:1019400011F0660F771F8091030290910402A0911D
:101950000502B09106029B01442737FD4095542FA4
:10196000820F931FA41FB51F80930302909304025C
:10197000A0930502B093060280910702909108029D
:10198000A0910902B0910A02820F931FA41FB51FF4
:101990008093070290930802A0930902B0930A0271
:1019A0008091030290910402A0910502B091060279
:1019B000815F9A4BA440B04064F080E393E9ABEFC1
:1019C000BFEF8093030290930402A0930502B093AB
:1019D00006028091030290910402A0910502B09149
:1019E000060280519544AB4FBF4F64F480ED9CE6F6
:1019F000A4E0B0E08093030290930402A093050258
:101A0000B093060280917800909179000F9710F4BE
:101A100068E17CEF8091780090917900079710F44D
:101A200060E378EF8091780090917900835F934034
:101A300010F068EE73E080917800909179008A5FF1
:101A4000934010F060ED77E08091B5019091B60180
:101A5000860F971F9093B6018093B5018091C001C6
:101A60008F5F8093C00182E0A1C060917800709187
:101A700079008091D7019091D801681B790B8091F2
:101A800000018A3011F0660F771F8091FB01909161
:101A9000FC01A091FD01B091FE019B01442737FD9F
:101AA0004095542F820F931FA41FB51F8093FB01F5
:101AB0009093FC01A093FD01B093FE018091FF0182
:101AC00090910002A0910102B0910202820F931F37
:101AD000A41FB51F8093FF0190930002A093010201
:101AE000B09302028091FB019091FC01A091FD0155
:101AF000B091FE01815F9A4BA440B04064F080E356
:101B000093E9ABEFBFEF8093FB019093FC01A093AF
:101B1000FD01B093FE018091FB019091FC01A09129
:101B2000FD01B091FE0180519544AB4FBF4F64F46D
:101B300080ED9CE6A4E0B0E08093FB019093FC0173
:101B4000A093FD01B093FE018091780090917900FF
:101B50000F9710F468E17CEF809178009091790004
:101B6000079710F460E378EF809178009091790006
:101B7000835F934010F068EE73E08091780090915D
:101B800079008A5F934010F060ED77E08091B301B7
:101B90009091B401860F971F9093B4018093B30185
:101BA0008091BF018F5F8093BF0184E08093CA0161
:101BB000C8C140910701509108018091780090912F
:101BC00079009A01220F331F240F351F63E070E064
:101BD0000E94A32C260F371F3695279536952795FB
:101BE000309308012093070186E0E0CF8091DF0168
:101BF0009091E0012091780030917900821B930B45
:101C000090939E0480939D048091B9019091BA01B4
:101C100020919D0430919E04820F931F9093BA01EE
:101C20008093B9018091C3018F5F8093C30187E0E6
:101C3000BDCF80917800909179002091DD013091A5
:101C4000DE01821B930B9093A9048093A8048091DA
:101C5000BB019091BC012091A8043091A904820F8E
:101C6000931F9093BC018093BB018091C2018F5F51
:101C70008093C2014093CA0186E0E4C0609178007D
:101C800070917900E090E101F090E2010091E301B0
:101C90001091E401882777FD8095982F0E94B62B3C
:101CA000A80197010E94102B0E94992B7093BE01EE
:101CB0006093BD012091BD013091BE01E0919D0472
:101CC000F0919E048091A8049091A90497FF03C00D
:101CD000909581959F4F64E070E00E94B72CEB01D6
:101CE000CF01F7FF03C0909581959F4F64E070E0AE
:101CF0000E94B72C260F371F2C0F3D1F3093BE01BB
:101D00002093BD018091BD019091BE01029704F125
:101D10006091E1017091E2018091E3019091E40111
:101D200020E030E048E454E40E94C02B88230CF00B
:101D30003CC06091E1017091E2018091E3019091DA
:101D4000E4012AE037ED43EA5CE30E94112B25C051
:101D50008091BD019091BE018F5F9F4F34F56091DE
:101D6000E1017091E2018091E3019091E40120E0B2
:101D700030E046E154E40E94C32B1816B4F460919D
:101D8000E1017091E2018091E3019091E4012AE088
:101D900037ED43EA5CE30E94102B6093E1017093FE
:101DA000E2018093E3019093E40181E08093C40118
:101DB00080917800909179009093A00480939F0483
:101DC0002091130230911402409115025091160295
:101DD0008091BD019091BE01AA2797FDA095BA2FD1
:101DE000280F391F4A1F5B1F2093130230931402E0
:101DF0004093150250931602E0901302F0901402E3
:101E00000091150210911602609113027091140254
:101E1000809115029091160220E034E040E050E0FD
:101E20000E94EC2CE21AF30A040B150BE092130249
:101E3000F0921402009315021093160283E080932F
:101E4000CA0187E08093C9017CC08091AD04909164
:101E5000AE042091780030917900820F931F909307
:101E6000AE048093AD048091A5048F5F8093A50498
:101E70008091A504853008F460C08091780090912D
:101E8000790090930E0180930D011092A50480912A
:101E9000A1049091A2042091AD043091AE04821B64
:101EA000930B20912F0230913002821B930B909361
:101EB000C6018093C5016091AD047091AE04E090BD
:101EC0000901F0900A0100910B0110910C01882783
:101ED00077FD8095982FA8019701220F331F441F8B
:101EE000551F2E0D3F1D401F511F620F731F841F72
:101EF000951F24E030E040E050E00E94EC2C20935D
:101F0000090130930A0140930B0150930C01209179
:101F1000A1043091A2048091090190910A01A0913D
:101F20000B01B0910C01281B390B30933002209328
:101F30002F021092AE041092AD041092CA011092BA
:101F4000C9018091CA0180937C008FEE80937A0052
:101F5000FF91EF91DF91CF91BF91AF919F918F91C1
:101F60007F916F915F914F913F912F911F910F91B1
:101F7000FF90EF900F900FBE0F901F901895CF938A
:101F8000DF93A3E0B0E00E94072D802DC82FDD274E
:101F9000C531D10508F02A97C7BD84E690E00E94BC
:101FA000EB0B80910D0190910E0182559340D0F47E
:101FB000C0E0D0E017C0C7BD82E390E00E94EB0B09
:101FC00085E591E09F938F931F920E94B7078091C0
:101FD0000D0190910E010F900F900F908458934037
:101FE00020F02196CA3FD10530F3A3E0B0E00C2EDB
:101FF0000E940F2DC093AA048CE291E00E94EB0B8B
:10200000DF91CF910895E9E1F1E080E2819391E0E1
:10201000E936F907D9F70895FF920F931F9380913E
:10202000CE01282F3327C90181709070682F882333
:1020300091F08091CF01882311F0815002C08091EE
:1020400069018093CF01E9E1F1E080E2819391E0C1
:10205000E936F907D9F7A9014270507021FF0DC088
:102060008091CF018F5F8093CF01E9E1F1E080E2C1
:10207000819391E0E936F907D9F7662321F0452BE2
:1020800011F01092CF0181E18093CD018091CF01B9
:1020900099279F938F9382ED93E09F938F9311E005
:1020A000F12EFF920E94B7070091CF010F900F9081
:1020B0000F900F900F90053009F4F8C1063090F49E
:1020C000023009F4C8C0033030F40023F1F00130CD
:1020D00009F07CC35DC0033009F412C1043009F07B
:1020E00075C361C1083009F4B9C2093038F406304B
:1020F00009F432C2073009F069C38DC2093009F40E
:10210000EAC20A3009F062C324C31092CD0180EC08
:1021100093E09F938F93FF920E94B70784E180938F
:10212000CD01209100018FE390E09F938F931F9248
:102130001F92822F6AE00E94972C892F99279F93E4
:102140008F93822F0E94972C99279F938F938DEACC
:1021500093E09F938F93FF920E94B70788E280934A
:10216000CD010E940B0299279F938F9380EA93E001
:102170009F938F93FF920E94B7078CE38093CD01CA
:1021800080E993E09F938F93FF920E94B707B4C0BA
:102190008091EB0480FF47C01092CD0180912F0207
:1021A000909130029F938F9381E893E09F938F9358
:1021B0000F930E94B70784E18093CD018091310293
:1021C000909132029F938F9382E793E09F938F9336
:1021D0000F930E94B70788E28093CD0180910D0193
:1021E00090910E019F938F9383E693E09F938F933B
:1021F0000F930E94B7078CE38093CD018091AA04CE
:1022000099279F938F9384E593E09F938F930F93E8
:102210000E94B7078DB79EB744960FB6F8949EBF3D
:102220000FBE8DBFD8C284E18093CD018DE493E0D1
:102230009F938F930F930E94B70788E28093CD01FD
:102240008FE393E09F938F930F930E94B7078DB70F
:102250009EB70696E2CF1092CD0185E393E09F935F
:102260008F93FF920E94B70784E18093CD01609124
:10227000E7017091E8018091E9019091EA0120E085
:1022800034E040E050E00E94EC2C5F934F933F938A
:102290002F9386E293E09F938F93FF920E94B7075C
:1022A00088E28093CD016091EF017091F0018091FF
:1022B000F1019091F20120E034E040E050E00E9412
:1022C000EC2C5F934F933F932F9387E193E09F9381
:1022D0008F93FF920E94B7078CE38093CD0180918A
:1022E0001702909118029F938F9388E093E09F9339
:1022F0008F93FF920E94B7078DB79EB746968DCFFA
:102300001092CD018091BB049091BC042091B9043E
:102310003091BA049F938F933F932F9388EF92E06D
:102320009F938F93FF920E94B70784E18093CD0122
:102330008091BF049091C0042091BD043091BE04EF
:102340009F938F933F932F9388EE92E09F938F9369
:10235000FF920E94B70788E28093CD018091C30469
:102360009091C4042091C1043091C2049F938F9333
:102370003F932F9388ED92E09F938F93FF920E945B
:10238000B7078CE38093CD018091C7049091C80476
:102390002091C5043091C6049F938F933F932F9350
:1023A00088EC92E07AC01092CD01E091E404FF271E
:1023B000EE0FFF1FE954FB4F20813181E091E304D0
:1023C000FF27EE0FFF1FE954FB4F808191813F9360
:1023D0002F939F938F9388EB92E09F938F93FF921D
:1023E0000E94B70784E18093CD01E091E604FF27C6
:1023F000EE0FFF1FE954FB4F20813181E091E5048E
:10240000FF27EE0FFF1FE954FB4F808191813F931F
:102410002F939F938F9388EA92E09F938F93FF92DD
:102420000E94B70788E28093CD01E091E804FF277E
:10243000EE0FFF1FE954FB4F20813181E091E7044B
:10244000FF27EE0FFF1FE954FB4F808191813F93DF
:102450002F939F938F9388E992E09F938F93FF929E
:102460000E94B7078CE38093CD01E091EA04FF2737
:10247000EE0FFF1FE954FB4F20813181E091E90409
:10248000FF27EE0FFF1FE954FB4F808191813F939F
:102490002F939F938F9388E892E09F938F93FF925F
:1024A0000E94B7078DB79EB74C96B7CE1092CD015C
:1024B0008AE792E09F938F93FF920E94B70784E18F
:1024C0008093CD012091D7013091D8018091B30143
:1024D0009091B4016091BF013F932F9377270E94A1
:1024E000B72C7F936F938BE692E09F938F93FF922D
:1024F0000E94B70788E28093CD012091D9013091E5
:10250000DA018091B5019091B6016091C0013F93CD
:102510002F9377270E94B72C7F936F938CE592E0DF
:102520009F938F93FF920E94B7078CE38093CD0116
:102530002091DB013091DC018091B7019091B801CD
:102540006091C1013F932F9377270E94B72C7F930F
:102550006F938DE492E056C01092CD0180E492E03A
:102560009F938F93FF920E94B70784E18093CD01E0
:102570002091DD013091DE018091BB019091BC0181
:102580006091C2013F932F9377270E94B72C7F93CE
:102590006F9381E392E09F938F93FF920E94B7071E
:1025A00088E28093CD012091DF013091E00180919C
:1025B000B9019091BA016091C3013F932F9377279E
:1025C0000E94B72C7F936F9382E292E09F938F9348
:1025D000FF920E94B7078CE38093CD016091E101E7
:1025E0007091E2018091E3019091E40100919F04D8
:1025F0001091A0040E94992B7F936F931F930F93C8
:1026000083E192E09F938F93FF920E94B7078DB76B
:102610009EB7489602CE84E18093CD018091070158
:10262000909108019F938F9384E092E09F938F9302
:10263000FF920E94B70788E28093CD018091270224
:1026400099279F938F9385EF91E09F938F93FF92AC
:102650000E94B7078DB79EB70A96DFCD1092CD01C5
:1026600086EE91E09F938F93FF920E94B70784E1DB
:102670008093CD0180911B0290911C029F938F93B8
:1026800087ED91E09F938F93FF920E94B70788E2B6
:102690008093CD0180911702909118029F938F93A0
:1026A00088EC91E09F938F93FF920E94B7078CE391
:1026B0008093CD018091190290911A029F938F937C
:1026C00089EB91E09F938F93FF920E94B7078DB79C
:1026D0009EB74296A2CD1092CD0180911F0290919B
:1026E00020029F938F938DEA91E09F938F93FF92A7
:1026F0000E94B70784E18093CD01809121029091DF
:1027000022029F938F9381EA91E09F938F93FF9290
:102710000E94B70788E28093CD01809123029091B7
:1027200024029F938F9385E991E09F938F93FF926B
:102730000E94B7078CE38093CD0180912502909190
:1027400026029F938F9389E891E09F938F93FF9246
:102750005FCD1092CD0181E891E09F938F93FF921E
:102760000E94B70784E18093CD0180918D01992764
:102770009F938F9383E791E09F938F93FF920E94A3
:10278000B70788E28093CD018091AE019091AF01AF
:102790009F938F9385E691E09F938F93FF920E9482
:1027A000B7078CE38093CD018091070599279F930C
:1027B0008F938091060599279F938F9387E591E0EA
:1027C0009F938F93FF920E94B70724CD01500093EF
:1027D00069011092CF011092CE011F910F91FF90CD
:1027E00008951092B9008AE28093B800089585EAAE
:1027F0008093BC0080E090E0089584E98093BC0061
:1028000008951092B9008093BB0085E88093BC00C6
:1028100080E090E008951F920F920FB60F9211245E
:102820008F939F93EF93FF938091D0018F5F80935D
:10283000D00181508330A9F1843028F4813091F0A7
:10284000823008F50AC0853089F18530B8F18630CC
:10285000A9F1873009F061C045C08091D101880F8E
:102860008E5A09C08091D1018F5F8093D101815030
:1028700027C0809170021092B9008093BB0085E858
:102880008093BC004AC084E98093BC008091D10150
:10289000843018F41092D00102C01092D10185EA60
:1028A000EFCF8091D201880F8D5AE5CF8091BB0088
:1028B000E091D201FF27E155FB4F80838091D20147
:1028C000813039F08130A8F2823031F0833029F53F
:1028D00006C080917102CFCF80917402CCCF8091DD
:1028E0007602C9CF8091D2019091BB00E82FFF27DB
:1028F000E155FB4F94838F5F8093D201843010F0B9
:102900001092D20184E98093BC008AE090E0909319
:102910007B0180937A011092D0018091BC00806885
:102920008093BC00FF91EF919F918F910F900FBE0C
:102930000F901F9018954CEB50E084E9DA018C93CE
:102940001092D0012BEB30E0F90180811092D1017F
:1029500080E88C931092BD001092BA001082E9EBCF
:10296000F0E01082A8EBB0E01C9210828AE28C9317
:1029700085EADA018C931082F901108285E88C9344
:10298000089583EC80938100EFE6F0E0808180621F
:1029900080831092DC011092DB011092DA01109218
:1029A000D9011092D8011092D70108951F920F9269
:1029B0000FB60F9211240F931F932F933F934F93B2
:1029C0005F936F937F938F939F93AF93BF93CF93B7
:1029D000DF93EF93FF9320918600309187008091E1
:1029E000D5019091D601281B390B809186009091DA
:1029F00087009093D6018093D501C9018D5D9540E4
:102A00008356994148F481E090E09093D4018093FB
:102A1000D30110926A0178C00091D3011091D401C2
:102A20000A3011050CF070C0C9018B5F9040845BC7
:102A3000914008F051C0E901CE50D240F801EE0FAC
:102A4000FF1FE954FB4F808191819E01281B390BA8
:102A5000C90137FF03C0909581959F4F06974CF4AD
:102A600080912702883C28F480912702865F80931A
:102A70002702F801EE0FFF1FE954FB4F208131813F
:102A8000C901880F991F820F931F8C0F9D1F64E04F
:102A900070E00E94B72CCE010196861797071CF4B0
:102AA0006150704006C021976C177D0714F46F5F6A
:102AB0007F4FF801EE0FFF1FDF01A954BB4F8D912F
:102AC0009C9111979B01281B390BE353FB4F3183DA
:102AD000208311967C936E93F8013196F093D40184
:102AE000E093D301E530F10519F45D9A5C980BC0D1
:102AF0005D98E630F10511F45C9A05C05C98379753
:102B000011F45B9A01C05B98FF91EF91DF91CF9137
:102B1000BF91AF919F918F917F916F915F914F91F5
:102B20003F912F911F910F910F900FBE0F901F900B
:102B30001895AF92BF92CF92DF92EF92FF920F93D0
:102B40001F9310927A008091BF01882369F08091D1
:102B5000B3019091B4016091BF0177270E94B72C17
:102B60007093200560931F058091C001882369F050
:102B70008091B5019091B6016091C00177270E94C4
:102B8000B72C70931E0560931D058091C1018823A9
:102B900069F08091B7019091B8016091C1017727E8
:102BA0000E94B72C70932C0560932B058091C20175
:102BB0008823D9F1E0902805F09029056091BB01A8
:102BC0007091BC012091C2010027F7FC0095102FE5
:102BD0005701680183E0AA0CBB1CCC1CDD1C8A9544
:102BE000D1F7AE18BF08C00AD10A882777FD8095B3
:102BF000982FB4E0660F771F881F991FBA95D1F7F9
:102C00003327442755270E94EC2CA20EB31EC41E66
:102C1000D51EC601B50128E030E040E050E00E943A
:102C2000EC2C30932905209328058091C30188233B
:102C3000D9F1E0903105F09032056091B9017091C1
:102C4000BA012091C3010027F7FC0095102F57010E
:102C50006801A3E0AA0CBB1CCC1CDD1CAA95D1F713
:102C6000AE18BF08C00AD10A882777FD8095982F33
:102C7000F4E0660F771F881F991FFA95D1F7332765
:102C8000442755270E94EC2CA20EB31EC41ED51E4D
:102C9000C601B50128E030E040E050E00E94EC2C95
:102CA00030933205209331058091C4018823A1F12E
:102CB000E0902205F09023056091BD017091BE0166
:102CC0002091C4010027F7FC0095102F57016801DF
:102CD000E3E0AA0CBB1CCC1CDD1CEA95D1F7AE18B6
:102CE000BF08C00AD10A882777FD8095982F33271F
:102CF000442755270E94EC2CA20EB31EC41ED51EDD
:102D0000C601B50128E030E040E050E00E94EC2C24
:102D100030932305209322051092B4011092B30141
:102D20001092BF011092B6011092B5011092C0012D
:102D30001092B8011092B7011092C1011092BA011D
:102D40001092B9011092C3011092BC011092BB0104
:102D50001092C2011092BE011092BD011092C401E6
:102D600080910B0290910C02A0910D02B0910E0285
:102D70008093F7019093F801A093F901B093FA01C1
:102D80008091FB019091FC01A091FD01B091FE01A9
:102D90008093E7019093E801A093E901B093EA01E1
:102DA0008091030290910402A0910502B091060265
:102DB0008093EF019093F001A093F101B093F201A1
:102DC0008091FF0190910002A0910102B091020256
:102DD0008093EB019093EC01A093ED01B093EE0191
:102DE0008091070290910802A0910902B0910A0215
:102DF0008093F3019093F401A093F501B093F60151
:102E00008FEE80937A0020911F02309120028091F2
:102E1000E704E82FFF27EE0FFF1FE954FB4F8081E7
:102E2000918182599F4F281739071CF42F5F3F4F1C
:102E30000CC08081918182599F4F821793074CF477
:102E40002115310531F0215030403093200220937C
:102E50001F0220912102309122028091E804E82F84
:102E6000FF27EE0FFF1FE954FB4F808191818259AC
:102E70009F4F281739071CF42F5F3F4F0CC08081EC
:102E8000918182599F4F821793074CF42115310588
:102E900031F02150304030932202209321022091C2
:102EA0002302309124028091E904E82FFF27EE0FDE
:102EB000FF1FE954FB4F8081918182599F4F281752
:102EC00039071CF42F5F3F4F0CC0808191818259DC
:102ED0009F4F821793074CF42115310531F0215093
:102EE0003040309324022093230220912502309118
:102EF00026028091EA04E82FFF27EE0FFF1FE95416
:102F0000FB4F8081918182599F4F281739071CF40C
:102F10002F5F3F4F0CC08081918182599F4F821754
:102F200093074CF42115310531F021503040309396
:102F300026022093250280911F029091200297FF84
:102F400005C01092200210921F020AC08F3F910507
:102F500039F034F08FEF90E09093200280931F02BD
:102F6000809121029091220297FF05C010922202C7
:102F7000109221020AC08F3F910539F034F08FEF93
:102F800090E09093220280932102809123029091FD
:102F9000240297FF05C010922402109223020AC057
:102FA0008F3F910539F034F08FEF90E09093240239
:102FB00080932302809125029091260297FF05C0FD
:102FC00010922602109225020AC08F3F910539F017
:102FD00034F08FEF90E090932602809325021F91AA
:102FE0000F91FF90EF90DF90CF90BF90AF9008953A
:102FF00010927A008091BF01882369F08091B3011B
:103000009091B4016091BF0177270E94B72C709313
:10301000200560931F058091C001882369F080918D
:10302000B5019091B6016091C00177270E94B72C3D
:1030300070931E0560931D058091C101882369F07E
:103040008091B7019091B8016091C10177270E94EA
:10305000B72C70932C0560932B058091C2018823B7
:10306000D1F06091BB017091BC012091C201882711
:1030700077FD8095982FF4E0660F771F881F991FC2
:10308000FA95D1F73327442755270E94EC2C30932B
:103090002905209328058091C3018823D1F06091F0
:1030A000B9017091BA012091C301882777FD8095FD
:1030B000982FE4E0660F771F881F991FEA95D1F7D4
:1030C0003327442755270E94EC2C30933205209358
:1030D00031058091C401882399F06091BD01709100
:1030E000BE012091C401882777FD8095982F332752
:1030F000442755270E94EC2C30932305209322056A
:103100001092B4011092B3011092BF011092B60157
:103110001092B5011092C0011092B8011092B7013F
:103120001092C1011092BA011092B9011092C3011C
:103130001092BC011092BB011092C2011092BE010C
:103140001092BD011092C4018FEE80937A002091FD
:103150001F02309120028091E704E82FFF27EE0F35
:10316000FF1FE954FB4F8081918182599F4F28179F
:1031700039071CF42F5F3F4F0CC080819181825929
:103180009F4F821793074CF42115310531F02150E0
:1031900030403093200220931F0220912102309171
:1031A00022028091E804E82FFF27EE0FFF1FE95469
:1031B000FB4F8081918182599F4F281739071CF45A
:1031C0002F5F3F4F0CC08081918182599F4F8217A2
:1031D00093074CF42115310531F0215030403093E4
:1031E0002202209321022091230230912402809117
:1031F000E904E82FFF27EE0FFF1FE954FB4F808102
:10320000918182599F4F281739071CF42F5F3F4F38
:103210000CC08081918182599F4F821793074CF493
:103220002115310531F02150304030932402209394
:10323000230220912502309126028091EA04E82F92
:10324000FF27EE0FFF1FE954FB4F808191818259C8
:103250009F4F281739071CF42F5F3F4F0CC0808108
:10326000918182599F4F821793074CF421153105A4
:1032700031F0215030403093260220932502809176
:103280001F029091200297FF05C010922002109219
:103290001F020AC08F3F910539F034F08FEF90E0A4
:1032A0009093200280931F0280912102909122022C
:1032B00097FF05C010922202109221020AC08F3F90
:1032C000910539F034F08FEF90E0909322028093D3
:1032D0002102809123029091240297FF05C0109251
:1032E0002402109223020AC08F3F910539F034F076
:1032F0008FEF90E090932402809323028091250227
:103300009091260297FF05C0109226021092250286
:1033100008958F3F910539F034F08FEF90E090934E
:1033200026028093250208951F938091EE048B3F1F
:1033300098F08B3F19F480911F020EC08C3F19F456
:103340008091210209C08D3F19F48091230204C0AD
:103350008E3F21F480912502809385018091850123
:10336000882319F41092850104C08F3F11F48093D3
:1033700085018091ED048B3F98F08B3F19F480918B
:103380001F020EC08C3F19F48091210209C08D3FAD
:1033900019F48091230204C08E3F21F4809125020C
:1033A0008093840180918401882319F41092840110
:1033B00005C0843618F084E6809384018091EF0480
:1033C0008B3F98F08B3F19F480911F020EC08C3F09
:1033D00019F48091210209C08D3F19F480912302D4
:1033E00004C08E3F21F48091250280938601809154
:1033F0008601882319F41092860105C0843618F0DE
:1034000084E6809386018091F1048B3F98F08B3F96
:1034100019F480911F020EC08C3F19F48091210293
:1034200009C08D3F19F48091230204C08E3F21F41E
:10343000809125028093870180918701882319F468
:103440001092870104C08F3F11F48093870180910F
:10345000F8048B3F98F08B3F19F480911F020EC047
:103460008C3F19F48091210209C08D3F19F480919D
:10347000230204C08E3F21F48091250280938801AD
:1034800080918801882319F41092880104C08F3F2D
:1034900011F4809388018091F9048B3F98F08B3F61
:1034A00019F480911F020EC08C3F19F48091210203
:1034B00009C08D3F19F48091230204C08E3F21F48E
:1034C0008091250280938901809189018B3010F4CD
:1034D0008AE002C08F3F11F4809389018091FA0441
:1034E0008B3F98F08B3F19F480911F020EC08C3FE8
:1034F00019F48091210209C08D3F19F480912302B3
:1035000004C08E3F21F48091250280938A0180912E
:103510008A01882319F410928A0104C08F3F11F4A4
:1035200080938A018091FF048B3F98F08B3F19F4C0
:1035300080911F020EC08C3F19F48091210209C0B6
:103540008D3F19F48091230204C08E3F21F48091B5
:10355000250280938C0180918C01882319F41092AC
:103560008C0104C08F3F11F480938C018091000581
:103570008B3F98F08B3F19F480911F020EC08C3F57
:1035800019F48091210209C08D3F19F48091230222
:1035900004C08E3F21F480912502809335028091F2
:1035A0003502882319F41092350204C08F3F11F4BC
:1035B00080933502809101058B3F98F08B3F19F481
:1035C00080911F020EC08C3F19F48091210209C026
:1035D0008D3F19F48091230204C08E3F21F4809125
:1035E00025028093360280913602882319F41092C6
:1035F000360204C08F3F11F4809336028091020599
:103600008B3F98F08B3F19F480911F020EC08C3FC6
:1036100019F48091210209C08D3F19F48091230291
:1036200004C08E3F21F4809125028093370280915F
:103630003702882319F41092370204C08F3F11F427
:1036400080933702809103058B3F98F08B3F19F4EC
:1036500080911F020EC08C3F19F48091210209C095
:103660008D3F19F48091230204C08E3F21F4809194
:1036700025028093380280913802882319F4109231
:10368000380204C08F3F11F48093380290910405F2
:103690009B3FB0F09B3F19F480911F0204C09C3FF8
:1036A00029F48091210280938D010CC09D3F19F473
:1036B00080912302F8CF9E3F29F480912502F3CF19
:1036C00090938D0180918D01882319F410928D01C2
:1036D00004C08F3F11F480938D019B3FB0F09B3F5E
:1036E00019F480911F0204C09C3F29F480912102AB
:1036F00080938D010CC09D3F19F480912302F8CF77
:103700009E3F29F480912502F3CF90938D01809103
:103710008D01882319F410928D0104C08F3F11F49C
:1037200080938D019B3FB0F09B3F19F480911F0265
:1037300004C09C3F29F48091210280938D010CC02C
:103740009D3F19F480912302F8CF9E3F29F4809188
:103750002502F3CF90938D0180918D01882319F478
:1037600010928D0104C08F3F11F480938D018091E0
:1037700009058B3F98F08B3F19F480911F020EC012
:103780008C3F19F48091210209C08D3F19F480917A
:10379000230204C08E3F21F48091250280938E0184
:1037A00080918E01882319F410928E0104C08F3FFE
:1037B00011F480938E0110918C01612F772767FDA2
:1037C0007095872F972F0E94B62B17FF06C020E019
:1037D00030E040E853E40E94112B27E137EB41ED44
:1037E00058E30E94302C6093800170938101809394
:1037F0008201909383018091F60480932A05809141
:10380000F504809321051F91089581E08093E304DE
:1038100032E03093E40483E08093E50424E02093D5
:10382000E60445E04093E70486E08093E80487E0FF
:103830008093E90488E08093EA041092EB048EE11F
:103840008093EC048BEF8093EE048AE08093EF0486
:1038500092E39093ED049093F1043093F00420935D
:10386000F2041092F30480E18093F4048FE08093DB
:10387000F5048AEF8093F6048AE18093F70480E8E8
:103880008093F8048FEA8093F9048093FA048EE51C
:103890008093FB0483E28093FC0484E18093FD0425
:1038A0001092FE041092FF04109200051092010580
:1038B000109202051092030584E68093040588E2C5
:1038C0008093050510920C059093060586E9809378
:1038D000070540930805909309058AE580930A053A
:1038E00010920B05A1E1B5E0EBE6F1E08CE0019070
:1038F0000D928150E1F7089581E08093E30482E026
:103900008093E40483E08093E50494E09093E604DC
:1039100045E04093E70486E08093E80487E08093E5
:10392000E90438E03093EA041092EB048EE18093CE
:10393000EC048BEF8093EE048AE08093EF0422E3A3
:103940002093ED042093F1049093F0049093F204FB
:103950003093F30480E18093F4048FE08093F504C6
:103960008AEF8093F6048AE18093F70480E88093DD
:10397000F80488E78093F90496E99093FA048EE5B9
:103980008093FB0483E28093FC0484E18093FD0434
:103990001092FE041092FF0410920005109201058F
:1039A000109202051092030584E68093040588E2D4
:1039B0008093050510920C0520930605909307054A
:1039C00040930805209309058AE580930A05109223
:1039D0000B05A1E1B5E0E3E7F1E08CE001900D9289
:1039E0008150E1F7089580912E02882301F510920D
:1039F00071021092700210927402109276028091FD
:103A00009A01882311F08093700280919B01882392
:103A100011F08093710280919C01882311F08093B2
:103A2000760280919D01882311F080937402809129
:103A300070029927909375048093740480917102A9
:103A40009927909377048093760480917602992742
:103A500090937904809378048091740299279093CD
:103A60007B0480937A041092D0011092D1010E94BD
:103A7000F7130895CF93DF931092DE011092DD01CA
:103A80001092E0011092DF0180E090E0A0E0B0E051
:103A90008093E1019093E201A093E301B093E401EC
:103AA0001092D8011092D7011092DA011092D90128
:103AB0001092DC011092DB010E94F81785E090E083
:103AC0000E94080BEC01CE010E94110B8823D9F350
:103AD0000E94F8178091EB0480FF10C080910D01C7
:103AE00090910E01875B934038F480910D01909185
:103AF0000E018E5E924010F40E94BF0F8091000173
:103B00008A3041F580911F059091200597FF03C0F1
:103B1000909581959F4F9093D8018093D701809184
:103B20001D0590911E0597FF03C0909581959F4FAD
:103B30009093DA018093D90180912B0590912C0507
:103B400097FF03C0909581959F4F9093DC018093E0
:103B5000DB0133C080911F059091200597FF03C0C2
:103B6000909581959F4F62E070E00E94B72C709312
:103B7000D8016093D70180911D0590911E0597FF94
:103B800003C0909581959F4F62E070E00E94B72C32
:103B90007093DA016093D90180912B0590912C05E7
:103BA00097FF03C0909581959F4F62E070E00E945F
:103BB000B72C7093DC016093DB018091310590910B
:103BC000320597FF03C0909581959F4F60E170E0AB
:103BD0000E94B72C7093E0016093DF01809128056B
:103BE0009091290597FF03C0909581959F4F60E1C3
:103BF00070E00E94B72C7093DE016093DD0160914C
:103C00009F047091A004882777FD8095982F0E94CB
:103C1000B62B6093E1017093E2018093E3019093EE
:103C2000E4011092FB011092FC011092FD01109230
:103C3000FE011092FF0110920002109201021092F8
:103C400002021092030210920402109205021092D6
:103C500006021092070210920802109209021092B6
:103C60000A0210920B0210920C0210920D02109296
:103C70000E021092200510921F0510921E05109240
:103C80001D0510922C0510922B0580910901909131
:103C90000A01A0910B01B0910C019093A2048093B2
:103CA000A1041092C6011092C50110921302109245
:103CB0001402109215021092160280911702909130
:103CC000180290931A02809319020E94D92A82E363
:103CD00090E09093AD018093AC01DF91CF91089576
:103CE0001F93182F0EC080912E02882361F484E662
:103CF00090E09093AD018093AC018AEF90E00E9438
:103D0000EB0B115080F71F9108952F923F924F9225
:103D10005F926F927F928F929F92AF92BF92CF925B
:103D2000DF92EF92FF920F931F93CF93DF93CDB764
:103D3000DEB724970FB6F894DEBF0FBECDBF0E944A
:103D40009915299AE091E504FF27EE0FFF1FE9542A
:103D5000FB4F4080518028E730E0420E531E57FE53
:103D600002C04424552480912702843608F05BC0A9
:103D700080910201882399F48091030190910401BC
:103D80008F5F9F4F61F488E99AE39093AD01809330
:103D9000AC0180E09CE0909304018093030180914A
:103DA000440290914502009731F0019790934502AB
:103DB0008093440204C010922E0210921D02809142
:103DC00000018A3011F4289A01C0289880913F029E
:103DD00090914002815D974018F18091FC04482E3B
:103DE000552481E080931D02E091E304FF27EE0F4C
:103DF000FF1FE954FB4F11821082E091E404FF277A
:103E0000EE0FFF1FE954FB4F11821082E091E60490
:103E1000FF27EE0FFF1FE954FB4F11821082CAC12A
:103E200010922E02C7C1809127028D3808F4C2C1BA
:103E300010921D028091FD0422E3829FC001112493
:103E4000909345028093440259E2451651046CF068
:103E500080913F02909140026FEF8F3F960781F172
:103E600001969093400280933F0280913F0290918F
:103E70004002883C910520F078E24716510404F591
:103E80001092560210925702109258021092590244
:103E90001092520210925302109254021092550244
:103EA00010920B0210920C0210920D0210920E0250
:103EB00010920F0210921002109211021092120230
:103EC00089EC481651040CF4D5C080912E02882349
:103ED00009F070C1E091E604FF27EE0FFF1FE954DF
:103EE000FB4F808191818C3491050CF4C0C080918E
:103EF00043028F5F80934302893C08F45BC1299899
:103F000010922E02109243021092400210923F0231
:103F10008091E304282F3327F901EE0FFF1FE954A6
:103F2000FB4F80819181873491059CF4E091E404FA
:103F3000FF27EE0FFF1FE954FB4F0190F081E02DAA
:103F4000F7FF03C0F095E195FF4FE734F1050CF45E
:103F50006CC08091E404682F7727DB01AA0FBB1F98
:103F6000A954BB4F8D919C911197873491053CF0DA
:103F7000F901EE0FFF1FE954FB4F808191818D9174
:103F80009C918734910564F0F901EE0FFF1FE9540D
:103F9000FB4F808191818734910514F042E001C08C
:103FA00041E0FB01EE0FFF1FE954FB4F808191813F
:103FB000863491055CF4F901EE0FFF1FE954FB4FC5
:103FC00080819181873491050CF043E0FB01EE0F75
:103FD000FF1FE954FB4F808191818A5B9F4F5CF406
:103FE000F901EE0FFF1FE954FB4F80819181873467
:103FF00091050CF044E0660F771F69547B4FFB017D
:10400000808191818A5B9F4F5CF4220F331F29547A
:104010003B4FD9018D919C91863491050CF445E07C
:10402000A2E0B0E0042E0E940F2D8091EB0480FFEF
:1040300010C080910D0190910E01875B934038F480
:1040400080910D0190910E018E5E924010F40E94BD
:10405000BF0F0E940B024AE363EE74E00E9432023B
:104060000E943A1D0E940B020E94701EA3C0109273
:104070004302A0C0F3E24F1651040CF09BC08091A4
:10408000E604482F5527FA01EE0FFF1FE954FB4FB6
:1040900080819181855B9F4F0CF06DC080914202C1
:1040A0008F5F80934202893C08F467C088EC80935C
:1040B000420281E090E09093400280933F0281E0D1
:1040C00080932E0210924E0210924F0210925002D4
:1040D0001092510210920B0210920C0210920D02DB
:1040E00010920E0210920F02109210021092110202
:1040F000109212021092FB011092FC011092FD012D
:104100001092FE0110920302109204021092050216
:10411000109206028091E7019091E801A091E901D7
:10412000B091EA018093FF0190930002A0930102F5
:10413000B09302028091EF019091F001A091F10102
:10414000B091F2018093070290930802A0930902B4
:10415000B0930A021092560210925702109258021F
:10416000109259021092520210925302109254026D
:104170001092550202C010924202440F551F49543A
:104180005B4FDA018D919C918C3491058CF080917C
:1041900041028F5F80934102893C60F010922E02B1
:1041A00088EC809341021092400210923F0202C0BC
:1041B0001092410280916A01815080936A0180913E
:1041C0006A018F3F29F080911D02882309F4BCC148
:1041D0000E949419E091E304FF27EE0FFF1FDF0117
:1041E000A954BB4F4D915C918091F204682E7724C5
:1041F000E353FB4F808191812091F3043327469D47
:104200005001479DB00C569DB00C1124FC01E29F5B
:10421000C001E39F900DF29F900D1124A80EB91ECE
:10422000B0922902A0922802E091E404FF27EE0F49
:10423000FF1FDF01A954BB4F4D915C91E353FB4F2E
:1042400080819181469D4001479D900C569D900C28
:104250001124AC01429FC001439F900D529F900DCD
:104260001124880E991E90922B0280922A02E091CE
:10427000E604FF27EE0FFF1FE954FB4F8081918179
:10428000909581959F4F90932D0280932C021091D1
:104290008901612F772767FD7095872F972F0E94DF
:1042A000B62B17FF06C020E030E040E853E40E9440
:1042B000112B20E030E040E251E40E94112B20E07D
:1042C00030E040E85BE30E94302C6B017C0160939E
:1042D0002D0570932E0580932F0590933005109136
:1042E0008A01612F772767FD7095872F972F0E948E
:1042F000B62B17FF06C020E030E040E853E40E94F0
:10430000112B20E030EE4BE257E40E94532B6093D8
:1043100024057093250580932605909327058091A9
:10432000EB0482FF0CC080E090E0A0E0B0E080935E
:10433000240590932505A0932605B093270520E03A
:1043400030E040E050E0C701B6010E94C02B882356
:1043500064F480E090E0A0E0B0E080932D059093BD
:104360002E05A0932F05B093300520E030E040E00B
:1043700050E060912405709125058091260590916B
:1043800027050E94C02B882364F480E090E0A0E021
:10439000B0E08093240590932505A0932605B09363
:1043A000270580910B05992782FDCEC083FDCCC0E7
:1043B0008091E7019091E801A091E901B091EA01B3
:1043C00081569A4EA040B04044F1C30173E0880F7B
:1043D000991F7A95E1F7A501481B590B50932902C3
:1043E000409328028091E7019091E801A091E901B2
:1043F000B091EA0181589843A140B0400CF43FC00D
:10440000C30164E0880F991F6A95E1F7481B590BB7
:10441000509329024093280232C08091E701909185
:10442000E801A091E901B091EA01805A9541AF4FAE
:10443000BF4F2CF5930153E0220F331F5A95E1F73C
:104440002A0D3B1D30932902209328028091E70119
:104450009091E801A091E901B091EA018158984357
:10446000A140B04064F0C30144E0880F991F4A9511
:10447000E1F7281B390B3093290220932802809101
:10448000EF019091F001A091F101B091F2018156FC
:104490009A4EA040B0403CF1C30133E0880F991F11
:1044A0003A95E1F7A401481B590B50932B02409316
:1044B0002A028091EF019091F001A091F101B09159
:1044C000F20181589843A140B0400CF43DC024E073
:1044D000660C771C2A95E1F74619570950932B0271
:1044E00040932A0231C08091EF019091F001A09198
:1044F000F101B091F201805A9541AF4FBF4F24F5C1
:10450000930193E0220F331F9A95E1F7280D391D8F
:1045100030932B0220932A028091EF019091F001B9
:10452000A091F101B091F20181589843A140B040AF
:104530005CF084E0660C771C8A95E1F72619370950
:1045400030932B0220932A028091E404E82FFF2766
:10455000EE0FFF1FE954FB4F2081318180910A0546
:10456000482F55274217530724F480910B0582FDED
:104570000DC02081318188279927841B950B28172E
:1045800039077CF480910B0583FF0BC081E0809399
:10459000340280910905682E77246414750424F090
:1045A00002C01092340232018091E304E82FFF2709
:1045B000EE0FFF1FE954FB4F808191814817590787
:1045C00024F480910B0580FD0DC020813181882766
:1045D0009927841B950B281739078CF480910B05BC
:1045E00081FF0DC081E080933302109234028091EC
:1045F000090599278615970524F43C0102C01092FD
:10460000330290901D02992041F110922D021092D8
:104610002C02109229021092280210922B02109262
:104620002A028DEC9CECACECBDE380932D059093BD
:104630002E05A0932F05B09330058AE097EDA3EAED
:10464000BBE38093240590932505A0932605B093A2
:10465000270510923402109233028091C701909185
:10466000C8018D54914008F498C02091EB0130911D
:10467000EC014091ED015091EE018091E7019091A4
:10468000E801A091E901B091EA01281B390B4A0B1E
:104690005B0BE090F301F090F4010091F5011091B3
:1046A000F6018091EF019091F001A091F101B0919C
:1046B000F201E81AF90A0A0B1B0B1092C8011092BA
:1046C000C701273A31054105510534F08091D701E2
:1046D0009091D80101960AC02A553F4F4F4F5F4F26
:1046E0004CF48091D7019091D80101979093D80113
:1046F0008093D70177EAE716F1040105110534F03C
:104700008091D9019091DA0101960EC08AE5E816F0
:104710008FEFF8068FEF08078FEF18074CF48091A2
:10472000D9019091DA0101979093DA018093D90130
:1047300010927A008091E7019091E801A091E9013F
:10474000B091EA018093FF0190930002A0930102CF
:10475000B09302028091EF019091F001A091F101DC
:10476000B091F2018093070290930802A09309028E
:10477000B0930A028091F7019091F801A091F9019C
:10478000B091FA0180930F0290931002A09311024E
:10479000B09312028FEE80937A002090240530901F
:1047A0002505409026055090270520E030E040E0A8
:1047B00050E0C201B1010E94C02B882309F4F7C068
:1047C00080913302882309F0F2C08091340288235B
:1047D00009F0EDC06091E7017091E8018091E90175
:1047E0009091EA012091F704A22EBB24CC24DD2471
:1047F000E0902805F0902905A60195010E94EC2C77
:104800000027F7FC0095102F2E193F09400B510B84
:1048100020934A0230934B0240934C0250934D0236
:104820008091280590912905AA2797FDA095BA2F78
:10483000B7FF07C0B095A095909581959F4FAF4F5A
:10484000BF4F883C9105A105B1053CF4CA01B901EF
:1048500028E030E040E050E006C0CA01B90120E1A4
:1048600030E040E050E00E94EC2C20934A0230936C
:104870004B0240934C0250934D026091EF017091B6
:10488000F0018091F1019091F201E0903105F090FA
:104890003205A60195010E94EC2C0027F7FC00953B
:1048A000102F2E193F09400B510B209346023093D5
:1048B00047024093480250934902809131059091FC
:1048C0003205AA2797FDA095BA2FB7FF07C0B0956C
:1048D000A095909581959F4FAF4FBF4F883C910514
:1048E000A105B1053CF4CA01B90128E030E040E07F
:1048F00050E006C0CA01B90120E130E040E050E0DC
:104900000E94EC2C209346023093470240934802C9
:104910005093490280914A0290914B02A0914C021F
:10492000B0914D02853FE1E09E07E0E0AE07E0E098
:10493000BE072CF084EF91E0A0E0B0E009C08C50FD
:104940009E4FAF4FBF4F64F48CE09EEFAFEFBFEFD1
:1049500080934A0290934B02A0934C02B0934D0275
:104960008091460290914702A0914802B09149027D
:10497000853F21E0920720E0A20720E0B2072CF05B
:1049800084EF91E0A0E0B0E009C08C509E4FAF4FA3
:10499000BF4FECF48CE09EEFAFEFBFEF8093460289
:1049A00090934702A0934802B093490210C010921E
:1049B0004A0210924B0210924C0210924D02109239
:1049C0004602109247021092480210924902109239
:1049D0007A008091FB019091FC01A091FD01B091C2
:1049E000FE0120914A0230914B0240914C025091BD
:1049F0004D02821B930BA40BB50B8093FB0190938C
:104A0000FC01A093FD01B093FE01809103029091FF
:104A10000402A0910502B091060220914602309155
:104A200047024091480250914902821B930BA40B0C
:104A3000B50B8093030290930402A0930502B093F8
:104A4000060200912C0210912D02A80117FF04C04C
:104A500044275527401B510B443251053CF08091AF
:104A6000EB0484FD03C081E080933B022091F404B9
:104A70003327049FC001059F900D149F900D1124B2
:104A8000AC01249FC001259F900D349F900D1124EF
:104A900060E072E00E94B72C7B01209FC001219F43
:104AA000900D309F900D112464E070E00E94B72CAF
:104AB000E60EF71EB701882777FD8095982F69834A
:104AC0007A838B839C8360934E0270934F02809312
:104AD00050029093510280910B0290910C02A09190
:104AE0000D02B0910E0229813A814B815C81821BBB
:104AF000930BA40BB50B80930B0290930C02A09325
:104B00000D02B0930E0280910B0290910C02A091C5
:104B10000D02B0910E02895A9146A040B04064F057
:104B200088EA91E6A0E0B0E080930B0290930C023B
:104B3000A0930D02B0930E0280910B0290910C0293
:104B4000A0910D02B0910E0288559E49AF4FBF4F04
:104B500064F488E59EE9AFEFBFEF80930B0290937A
:104B60000C02A0930D02B0930E028FEE80937A0098
:104B70008091170290911802892B09F4A1C08091AD
:104B8000EB0483FF9DC06091E7017091E801809183
:104B9000E9019091EA0120E032E040E050E00E941B
:104BA000EC2C890137FF03C0109501951F4F6091D0
:104BB000EF017091F0018091F1019091F20120E0FC
:104BC00032E040E050E00E94EC2CB90137FF03C016
:104BD000709561957F4F601771070CF4B8016931CA
:104BE0007105A4F480913B02882381F08091390201
:104BF00090913A02892B51F48091170290911802FA
:104C000090931A028093190210923B02209188011E
:104C10003327629FC001639F900D729F900D1124F6
:104C200060E470E00E94B72CA901461B570B1416D4
:104C300015060CF03FC010927A0020913902309195
:104C40003A022115310561F500910B0210910C0219
:104C500020910D0230910E0280911B0290911C0256
:104C6000BC01649FC001659F900D749F900D11243D
:104C700060E270E00E94B72C882777FD8095982F1E
:104C8000060F171F281F391F00930B0210930C02E9
:104C900020930D0230930E028FEE80937A0010C0A5
:104CA0008FEE80937A002150304030933A02209367
:104CB000390206C084EF91E090933A028093390262
:104CC00080913C02815080933C028F3F09F062C08A
:104CD00081E380933C026091E7017091E80180914B
:104CE000E9019091EA01E090F704FF2400271127E1
:104CF000A80197010E94EC2C30935D0420935C0482
:104D00006091EF017091F0018091F1019091F201B9
:104D1000A80197010E94EC2C30935F0420935E045D
:104D200080912805909129059093610480936004F7
:104D300080913105909132059093630480936204D1
:104D400080912B0590912C059093650480936404C9
:104D500080912F02909130029093670480936604B3
:104D600060911302709114028091150290911602C5
:104D700020E032E040E050E00E94EC2C30936904E7
:104D800020936804809117029091180290936D040B
:104D900080936C04809133028823A9F060911F05F1
:104DA00070912005882777FD8095982F0E94B62B5B
:104DB00020912D0530912E0540912F055091300501
:104DC0000E94302C2CC06091E7017091E801809125
:104DD000E9019091EA01E0901F05F09020050E9402
:104DE000B62BA20191010E94302C5B016C010027BF
:104DF000F7FC0095102FC801B7010E94B62B209137
:104E00002D0530912E0540912F05509130050E94BF
:104E1000302C9B01AC01C601B5010E94112B0E94F0
:104E2000992B7093200560931F058091340288238D
:104E3000A9F060911D0570911E05882777FD80956A
:104E4000982F0E94B62B20912D0530912E05409170
:104E50002F05509130050E94302C2CC06091EF013D
:104E60007091F0018091F1019091F201E0901D05A7
:104E7000F0901E050E94B62BA20191010E94302CD9
:104E80005B016C010027F7FC0095102FC801B701EA
:104E90000E94B62B20912D0530912E0540912F05B3
:104EA000509130050E94302C9B01AC01C601B50128
:104EB0000E94112B0E94992B70931E0560931D0573
:104EC00060912B0570912C05E090F701F090F801AE
:104ED0000091F9011091FA01882777FD8095982FAC
:104EE0000E94B62B20912D0530912E0540912F0563
:104EF000509130050E94302C5B016C01C801B70154
:104F00000E94B62BA20191010E94302C20E030E0DB
:104F100040E05FE30E94302C9B01AC01C601B5016B
:104F20000E94112B0E94992B70932C0560932B05E6
:104F300080911F05909120058150984034F080E0C9
:104F400098E09093200580931F0580911F05909114
:104F500020058050984F34F480E098EF909320051E
:104F600080931F0580911D0590911E0581509840EA
:104F700034F080E098E090931E0580931D058091A9
:104F80001D0590911E058050984F34F480E098EFF5
:104F900090931E0580931D0580912B0590912C0503
:104FA0008150984034F080E098E090932C058093F5
:104FB0002B0580912B0590912C058050984F34F44F
:104FC00080E098EF90932C0580932B058091EB0463
:104FD000992780FFBCC02091850181FF0EC022333C
:104FE000B0F480912F029091300244979093320256
:104FF0008093310210921E020DC08091F004289F10
:10500000C00111244497909332028093310281E0D1
:1050100080931E02992021F01092320210923102E8
:1050200020912F0230913002409131025091320292
:10503000421753070CF08BC080911E02882309F49D
:1050400086C0241B350B809186019927AC01249FD3
:10505000C001259F900D349F900D112460E170E0F8
:105060000E94B72C8301061B170B2091C5013091BC
:10507000C601809184019927BC01269FC001279F0A
:10508000900D369F900D112468E070E00E94B72CBF
:10509000061B170B60911302709114028091150288
:1050A0009091160220E032E040E050E00E94EC2CAB
:1050B000CA01B901209187013327442755270E944F
:1050C000782C20E230E040E050E00E94EC2C7FEFB2
:1050D0002E3C370714F42EEC3FEF80913D02909167
:1050E0003E02AC01B4E0440F551FBA95E1F7481BEE
:1050F000590B2333310514F022E330E0021B130B6C
:10510000CA01800F911F60E170E00E94B72C70937C
:105110003E0260933D028091EC049927681779075D
:105120003CF4681679065CF090933E0280933D0251
:1051300080913D0290913E026816790624F47092A7
:105140003E0260923D0260903D0270903E0270927D
:105150006B0460926A0480902B0590902C058981E5
:105160009A81881A990AB301882777FD8095982F2C
:105170000E94B62B5B016C0123E333E343EB5FE357
:105180000E94302C7B018C01B401882777FD80952B
:10519000982F0E94B62BA80197010E94C32B1816C6
:1051A0002CF4C801B7010E94992B4B0123E333E390
:1051B00043EB5FEBC601B5010E94302C7B018C01F3
:1051C000B401882777FD8095982F0E94B62BA801FF
:1051D00097010E94C02B88232CF4C801B7010E94BC
:1051E000992B4B019AE06916710414F488249924D0
:1051F00020907C0130907D0140907E0150907F0195
:1052000060911F057091200520912802309129029C
:1052100040915A0250915B02241B350B621B730BA9
:10522000882777FD8095982F0E94B62B9B01AC01B3
:10523000C201B1010E94302C0E94992B709373021D
:105240006093720280917202909173028C01222706
:1052500017FD2095322F8091560290915702A09110
:105260005802B0915902080F191F2A1F3B1F0093C3
:105270005602109357022093580230935902101689
:10528000110612061306ACF4C80117FF03C090956F
:1052900081959F4F60E071E00E94B72C6F5F7F4F58
:1052A000882777FD8095982F061B170B280B390B45
:1052B00014C0C80117FF03C0909581959F4F60E00F
:1052C00071E00E94B72C6F5F7F4F882777FD809534
:1052D000982F060F171F281F391F0093560210938F
:1052E00057022093580230935902809156029091B0
:1052F0005702A0915802B09159028138EEE39E07FF
:10530000E0E0AE07E0E0BE072CF080E89EE3A0E01E
:10531000B0E009C08058914CAF4FBF4F64F480E8B3
:1053200091ECAFEFBFEF8093560290935702A0939A
:105330005802B093590220917202309173027301A6
:10534000EE0CFF1CC7012E153F050CF4C901CC243F
:10535000DD24CE18DF08B601C816D9060CF4BC014E
:105360009301280D391D260F371F37FF03C040E07A
:1053700050E008C080912A05482F5527241735078B
:105380000CF4A90180912105A82EBB24C501A41607
:10539000B5060CF4CA01809370029301261B370BEB
:1053A000280D391D37FF03C080E090E007C08091D1
:1053B0002A059927281739070CF4C9019501A81661
:1053C000B9060CF49C012093710260911D05709147
:1053D0001E0520912A0230912B0240915C025091CF
:1053E0005D02241B350B621B730B882777FD8095AC
:1053F000982F0E94B62B9B01AC01C201B1010E9403
:10540000302C0E94992B70936F0260936E028091F2
:105410006E0290916F028C01222717FD2095322F8A
:105420008091520290915302A0915402B091550282
:10543000080F191F2A1F3B1F00935202109353029B
:1054400020935402309355021016110612061306CB
:10545000ACF4C80117FF03C0909581959F4F60E0A1
:1054600071E00E94B72C6F5F7F4F882777FD809592
:10547000982F061B170B280B390B14C0C80117FFF8
:1054800003C0909581959F4F60E071E00E94B72C1A
:105490006F5F7F4F882777FD8095982F060F171F26
:1054A000281F391F00935202109353022093540275
:1054B000309355028091520290915302A091540270
:1054C000B091550281382EE3920720E0A20720E038
:1054D000B2072CF080E89EE3A0E0B0E009C080585D
:1054E000914CAF4FBF4F64F480E891ECAFEFBFEF4A
:1054F0008093520290935302A0935402B0935502AA
:1055000080916E0290916F0297018E159F050CF4A9
:105510009C01B601C216D3060CF4B9019301260F03
:10552000371F2819390937FF03C040E050E008C091
:1055300080912A05482F5527241735070CF4A90117
:105540009501A416B5060CF49A0120937602661A0A
:10555000770AB3016819790977FF03C020E030E0CA
:1055600008C080912A05282F3327621773070CF48F
:105570009B01C501A216B3060CF4C9018093740205
:1055800024960FB6F894DEBF0FBECDBFDF91CF914A
:105590001F910F91FF90EF90DF90CF90BF90AF9051
:1055A0009F908F907F906F905F904F903F902F9043
:1055B000089580915E0290915F02A0916002B09187
:1055C00061028093660290936702A0936802B09391
:1055D00069028091620290916302A0916402B0918D
:1055E000650280936A0290936B02A0936C02B09361
:1055F0006D02089510925B0210925A0210925D02A1
:1056000010925C020895FC014150504030F001902E
:105610000616D1F73197CF01089588279927089565
:105620005058192EEFD001D0D2C0BA1762077307B5
:1056300084079507B1F188F40EF410940B2EBA2F5D
:10564000A02D062E622F202D072E732F302D082E11
:10565000842F402D092E952F502DFF275523B9F06B
:10566000591B49F0573E98F0469537952795A795D1
:10567000F0405395C9F776F0BA0F621F731F841F6D
:1056800030F4879577956795B795F040939517FA1D
:105690000F2E0895BF1BBB27BA0B620B730B840B35
:1056A000F6CFDEF6DBC0AED001D091C0552359F065
:1056B000992369F09F575F57951B33F442F4903854
:1056C00011F4915805C09BC091589F3F09F4C6C082
:1056D000BB27112462177307840730F4660F771F06
:1056E000881FBB1F915098F311D00F920FD00F92CB
:1056F0000DD0A0E82617370748071B0609F0A04879
:10570000BA2F602D7F918F9100240895A0E8002486
:10571000621773078407B10528F0621B730B840BB3
:10572000B1090A2A660F771F881FBB1FA69581F74C
:10573000089597FB73D09F3738F0FEE9F91B982F37
:10574000872F762F6B2F05C086C096958795779506
:105750006795F150D0F73EF49095809570956195DE
:105760007F4F8F4F9F4F0895E89403C097FB0EF42F
:10577000F3DFB62F672F782F892F9EE9002427C0EB
:105780000ED05EF004C00BD026F001C008D019F096
:1057900020F48FEF089580E0089581E0089597FB4D
:1057A000092E052600F8689430D0E89407FC07C05D
:1057B000621773078407950721F008F40094079493
:1057C000989408959A95BB0F661F771F881F112420
:1057D0009923A1F08823B2F79F3F59F0BB0F48F4FB
:1057E00021F4002011F460FF04C06F5F7F4F8F4FE2
:1057F0009F4F881F9795879597F908952CC09FEF25
:1058000080EC0895052E092607FA440F551F5F3FC7
:1058100079F0AA27A51708F051E04795880F991F3E
:105820009F3F31F0BB27B91708F091E087950895A5
:105830009F919F911124E3CF97FB880F991F9F3F62
:1058400031F0BB27B91708F091E0879508959F9133
:105850009F911124D4CF6627772788279927089509
:10586000D1DF01D0B4CF992339F0552329F09F57C8
:105870005F57950F13F49AF1F1CF91589F3FE1F3E1
:10588000629FA12D0F92BB27639FA00DB11DEE2734
:10589000729FA00DB11DEE1FAF93AA27649FB00D9C
:1058A000E11D739FB00DE11DAA1F6627829FB00DF9
:1058B000E11DA61F5527749FE00DA11D551F839F55
:1058C000E00DA11D561F849FA00D511D852F7A2F1D
:1058D0006E2F1F900F9088231AF4939539F48FCF71
:1058E000000C111CBB1F661F771F881F012808951D
:1058F000629FD001739FF001829FE00DF11D649FB4
:10590000E00DF11D929FF00D839FF00D749FF00D3F
:10591000659FF00D9927729FB00DE11DF91F639FE0
:10592000B00DE11DF91FBD01CF0111240895991B90
:1059300079E004C0991F961708F0961B881F7A9586
:10594000C9F780950895AA1BBB1B51E107C0AA1F88
:10595000BB1FA617B70710F0A61BB70B881F991F10
:105960005A95A9F780959095BC01CD01089597FBB4
:10597000092E07260AD077FD04D0E5DF06D00020E7
:105980001AF4709561957F4F0895F6F7909581957B
:105990009F4F0895A1E21A2EAA1BBB1BFD010DC04B
:1059A000AA1FBB1FEE1FFF1FA217B307E407F507CF
:1059B00020F0A21BB30BE40BF50B661F771F881FAB
:1059C000991F1A9469F760957095809590959B0141
:1059D000AC01BD01CF01089597FB092E05260ED01D
:1059E00057FD04D0D7DF0AD0001C38F450954095FD
:1059F000309521953F4F4F4F5F4F0895F6F79095A3
:105A00008095709561957F4F8F4F9F4F0895F999BD
:105A1000FECFB2BDA1BDF89A119600B40895F999D0
:105A2000FECFB2BDA1BD00BC11960FB6F894FA9A94
:085A3000F99A0FBE0895FFCFA3
:105A38000A0164FFFF0A016400007D0000FF030102
:105A480002030405060708090A48616C6C6F2057B1
:105A5800656C7400000000000000000000000000F9
:105A6800000000000000000000000000000000002E
:105A7800000000000000000000000000000000001E
:105A8800000000000000000000000000000000000E
:105A98000000000000000000000A014B616D657203
:105AA80061000053706F7274000064000000803F52
:105AB80017B7D13830FB103A409696020A64460070
:00000001FF
